:10000000FE28A2008417800484138E010C1C8E002D
:1000100010200319F92810200319F9281020F928B5
:1000200022088E0601308C008D01000822050E0684
:10003000031D08008C0A03198D0F152808000408F9
:100040009200240884008030A1050830930003103A
:100050000318A10A3920920C930B28280000971A44
:10006000210C3920FC20031439201B088F001A08AA
:100070008C288413971F482800082204171F220683
:100080008000841700082204031C220680005328E5
:1000900000082204031C2206171B22068000841776
:1000A00022098005532817081F39FF3E8D001608C6
:1000B000F53E03188D0A00009928A11315080319AD
:1000C000A1170530940027308F00103073200330C3
:1000D0008F00E83073208F01643073208F010A3065
:1000E000732010087A288E0011088D0010088C00EB
:1000F000D8200C088C0094030319A11315080319C8
:1001000084281402031808000C08031DA113A11B66
:100110000800303EF4288F018E00FF308E07031C4C
:100120008F07031CF92803308D00DF3099208D28BC
:100130008D01E83E8C008D09FC30031CA2288C0741
:1001400003189F288C0764008D0F9F280C18A8287F
:100150008C1CAC280000AC280800013E93000A303B
:100160008E008F01D820930BB228100808008E0053
:100170000130BA2894000F080D02031DC1280E0893
:100180000C02043003180130031902301405031D5A
:10019000FF30F9288E000C08920010088C0012081D
:1001A00090000D08920011088D0012089100DA28C5
:1001B00091019001103092000D0D900D910D0E08DF
:1001C00090020F08031C0F0F91020318EE280E086F
:1001D00090070F0803180F0F910703108C0D8D0D5A
:1001E000920BDC280C08F92884001D088A001C08E2
:1001F00082008313031383126400080083168501B1
:100200001330860083128501860106298501860147
:1002100086128316861283128C0105308400013009
:1002200001200C08AC000D08AD002C088C002D0836
:100230008D00FD308F00E830B720031D0829861699
:10024000831686128312C030A8006A30A9002D08D8
:100250008F002C08CA20AA000D08AB002A088C00C9
:100260002B088D000030AD20A800A9012A088C00C1
:100270002B088D000A308E008F01D820AA000D08AF
:10028000AB000630A4000230A20054309600970163
:100290009A019B0195012A0890002B0891001F30BC
:1002A0009C009D015D202E302020950128089000A3
:1002B000290891001F309C009D015D202C302020DA
:1002C0004B3020206D3020202F302020683020201F
:1002D0002C30202095012C0890002D0891001F3013
:1002E0009C009D015D20303020202C302020753076
:1002F00020205330202045302020433020200D3056
:0C03000020200A302020082963008429F6
:02400E00F53F7C
:00000001FF
